:020000040000FA
:06000000703002303A28C6
:08000800A000030EA100831209
:1000100081018B100B11210E8300A00E200E090010
:0C007400203084008001840A80300402E7
:10008000031C3C281230B000412183160C3085053A
:1000900087018312850187010730990000309A009B
:1000A000103083168E008312603083168F00831207
:1000B0000030831691009F008312C83083168100A0
:1000C000831231309000003083168C008312103080
:1000D0008B00831600309B001C141A088312BC008E
:1000E000831610309B001C141A088312BD007E2159
:1000F00081018E018F010B118B100B108C018B175E
:100100009420311996202321B30B922803108519CE
:100110000314B90DF0303902031987210F30390269
:10012000031983218B218028640008000800311105
:100130000130B7008B132030370783169B001C1447
:100140001A088312A4001030370783169B001C1472
:100150001A088312A3000030370783169B001C1473
:100160001A088312A2008B17321CBC2822090339FB
:10017000A200A309A409A50901303702031DC5285F
:100180003D18C5283D143E14572101303702031D88
:10019000CE283D1CCE283D103E147B21CF28B70A27
:1001A00002303702031808009A280130B600B30065
:1001B000B400B500B70085018701B1139420B30BDB
:1001C000FB28031085190314B90DF0303902031907
:1001D0001929B41F8501B41F8701B40BFB28370808
:1001E000B6080319B6000319F928FF308500870007
:1001F000B6039630B400311DDE283111321C0529BA
:100200002D090339AD00AE09AF098B132030370734
:10021000BB002F08BA002C2110303707BB002E0876
:10022000BA002C2100303707BB002D08BA002C2162
:100230008B1785018701B70AB60102303702031C0C
:10024000DE287E2108003E1C08003E101030BB0056
:100250003D08BA002C2108008B133A0883161C15A0
:100260009A0083123B0883169B0055309D00AA30EC
:100270009D009C1464009C183A291C1183128B1752
:100280000800831620309B001C141A088312DF001C
:10029000FF30D5000230D6000C30D700BA30D8007D
:1002A0003730D900DA30DA006F30DB000800013077
:1002B000BD000430C200C5000530C400C600CA003D
:1002C0000730C100C300C700C800C9005F19C117CB
:1002D0005F19C2175F19C317DF19C4175F1AC51753
:1002E0005F1AC6175F1AC7175F1AC8175F1BC917AF
:1002F000DF18CA170800850187010800BD013D14F9
:100300003D18572108003D143E14572108003D10A8
:100310003E147B21080001303D05031908005F19D8
:1003200093295C1805165F199729DC1885165F1943
:100330009B295C190514DF199F29DC1985145F1AA4
:10034000A3295C1A87145F1AA729DC1A07155F1AFC
:10035000AB295C1B07145F1AAF29DC1B87165F1BD8
:10036000B3295D180716DF18B729DD188715E630A1
:100370000E02031CCF295F1D05165F1D85165F1D2C
:100380000514DF1D85145F1E87145F1E07155F1E91
:1003900007145F1E87165F1F0716DF1C87158F085F
:1003A000031908008F01850187015508DE00CD2360
:1003B000D5005608DE00CD23D6005708DE00551CB8
:1003C000CD23D7005808DE00D51CCD23D80059080E
:1003D000DE00551DCD23D9005A08DE00D51DCD23E2
:1003E000DA005B08DE00551ECD23DB005F1D122AFC
:1003F000C11B0D2AC11C0512C11C012A0512581966
:100400000516CB0B232A5608CB00C101D51BC114FE
:10041000D81BC1105818C110232A0512CB0B232A50
:10042000C103232AC108031905160319232ACB0B7C
:10043000232AD51BC1035508CB00D5185C14D51E43
:100440005C10D51D5C105F1D3F2AC21B3A2AC21CDE
:100450008512C21C2E2A851258188516CC0B502ADC
:100460005608CC00C201D61BC2145A18C210D619A5
:10047000C210502A8512CC0B502AC203502AC2083F
:10048000031985160319502ACC0B502AD61BC20318
:100490005608CC00D61ADC14561DDC10561FDC1092
:1004A0005F1D6C2AC31B672AC31C0510C31C5B2A73
:1004B00005105A190514CD0B7D2A5708CD00C3012C
:1004C000D71BC314D51AC310D719C3107D2A051022
:1004D000CD0B7D2AC3037D2AC30803190514031914
:1004E0007D2ACD0B7D2AD71BC3035708CD00571A91
:1004F0005C15571F5C11D71D5C11DF1D992AC41BA9
:10050000942AC41C8510C41C882A8510D51B851408
:10051000CE0BB52A5808CE00C401D81BC414D71A74
:10052000C410D819C410B52A8510CE0BB52AC4033F
:10053000B52ADF1FA42ACE0BB52A5808CE00D51B3A
:10054000DC15DA1FDC11B52AC40803198514031958
:10055000B52ACE0BB52AD81BC4035808CE00581AAA
:10056000DC15D81FDC11D81DDC115F1ED12AC51B7C
:10057000CC2AC51C8710C51CC02A8710D51A871421
:10058000CF0BE22A5908CF00C501D91BC514561A52
:10059000C510D81BC510E22A8710CF0BE22AC5036D
:1005A000E22AC508031987140319E22ACF0BE22AAD
:1005B000D91BC5035908CF00D91B5C16D91F5C1283
:1005C000D91C5C125F1EFE2AC61BF92AC61C071125
:1005D000C61CED2A0711D71A0715D00B0F2B5A0886
:1005E000D000C601DA1BC614D51AC610D619C6101B
:1005F0000F2B0711D00B0F2BC6030F2BC6080319A7
:10060000071503190F2BD00B0F2BDA1BC6035A0843
:10061000D0005A1ADC165A1EDC12DA1FDC125F1EDA
:100620002B2BC71B262BC71C0710C71C1A2B071008
:1006300059190714D10B3C2B5B08D100C701DB1BF8
:10064000C714D719C710DB19C7103C2B0710D10BE3
:100650003C2BC7033C2BC7080319071403193C2B79
:10066000D10B3C2BDB1BC7035B08D100DB195C17EC
:10067000DB1D5C135B1E5C135F1E582BC81B532BCA
:10068000C81C8712C81C472B871258198716D20B13
:10069000692B5608D200C801D91BC8145A19C810B2
:1006A000551AC810692B8712D20B692BC803692B06
:1006B000C808031987160319692BD20B692BD71B9E
:1006C000C8035908D200561ADC17561EDC13DA1F6D
:1006D000DC135F1F852BC91B802BC91C0712C91C8B
:1006E000742B071255190716D30B9F2B5808D300EC
:1006F000C901D61BC914D91AC910D819C9109F2B02
:100700000712D30B9F2BC9039F2B5F1C902BD30B7E
:100710009F2B5708D300D61B5D14D81F5D109F2B4D
:10072000C9080319071603199F2BD30B9F2BD51A42
:10073000C9035808D300D61B5D14D81F5D10DF1CF9
:10074000BB2BCA1BB62BCA1C8711CA1CAA2B87112C
:10075000D51B8715D40B08005508D400CA01D51B3A
:10076000CA14561ACA10D619CA1008008711D40B19
:100770000800CA030800CA080319871503190800EE
:10078000D40B0800D81BCA035608D400591ADD142C
:10079000591EDD10DA1FDD100800C001DE08031944
:1007A000DE035E184014DE1A40144008C0015E1CCF
:0E07B0004014DE1E4014C005C00C5E0C080094
:084000000D000300040008009C
:02400E00CC33B1
:10420000FF00FF00FF00FF00FF00FF00FF00FF00B6
:10421000FF00FF00FF00FF00FF00FF00FF00FF00A6
:104220000100FF00FF00FF00FF00FF00FF00FF0094
:10423000FF00FF00FF00FF00FF00FF00FF00FF0086
:104240000300FF00FF00FF00FF00FF00FF00FF0072
:10425000FF00FF00FF00FF00FF00FF00FF00050060
:10426000FF00FF00FF00FF00FF00FF00FF00FF0056
:10427000FF00FF00FF00FF00FF00FF00FF00FF0046
:10428000FF00FF00FF00FF00FF00FF00FF00FF0036
:10429000FF00FF00FF00FF00FF00FF00FF00FF0026
:1042A000FF00FF00FF00FF00FF00FF00FF00FF0016
:1042B000FF00FF00FF00FF00FF00FF00FF00FF0006
:1042C000FF00FF00FF00FF00FF00FF00FF00FF00F6
:1042D000FF00FF00FF00FF00FF00FF00FF00FF00E6
:1042E000FF00FF00FF00FF00FF00FF00FF00FF00D6
:1042F000FF00FF00FF00FF00FF00FF00FF000000C5
:00000001FF
